:020000040000FA
:1000000005280000000000008B1397018501860180
:100010008B01A701A801A901AA01AC0107309F002B
:10002000831603136730810030308500C8308600A6
:10003000831203139920D321A920861D202806119D
:100040008614E121E12107308101A5018E0106140A
:10005000831603130614831203134E20831603130F
:100060000610831203136520AA012508A9000108C0
:10007000A800A7016121861006152C1C46286C20BB
:10008000BB20B420C420832199214828EE20D3210D
:10009000E921CC21CC21CC212C141B28A2019330A6
:1000A00086192730A300A30F56285E286520A20FCB
:1000B0005628F930A200A20F5B285328AF308619CA
:1000C0005730A200A20F622808000B1D6A28A50A5B
:1000D0000B11080000000800861974212621093040
:1000E000BA00AB01393084003A08063C031D7A2877
:1000F0002B14AB142B1883280008003C031D832805
:100100002030132194282B14861D8A283A08013C9C
:10011000031908003030BC0000083C071321AB1C59
:1001200094282E301321AB10BA0B972808008403B3
:100130007428861202300D2102300D210C300D2161
:1001400000300D210C300D2100300D2106300D2125
:100150000800861200300D2101300D2108300D21DC
:1001600000300D218616080086120C300D2100305B
:100170000D2186160800203013214D301321483000
:1001800013217A30132108004230132161301321EA
:100190006E301321643013213A301321861DD92883
:1001A00055301321483013214630132120301321BC
:1001B000080056301321D228493013216E30132104
:1001C000743013213A301321080045301321783060
:1001D0001321743013213A301321080048301321C1
:1001E000493013212030132164301321653013214D
:1001F00020301321573013214E3013213230132178
:100200004130132120301321763013213630132151
:100210002E3013213230132108008500E12106160B
:10022000E12106120800C000BC00BD003C0E0F39E1
:100230008500DD210616DD2106123D080F398500F7
:10024000DD210616DD210612FC2108002030BB004E
:100250000930BA00313084008001BA0B30293229CC
:10026000840A2C2950213721BB0B32290800273062
:1002700084000310800D840A800D840A800D840A96
:10028000800D0930BA0031308400800D0310001A4F
:1002900003140F308005BA0B4E290800840A452943
:1002A0000930BA00313084000008A200043C031871
:1002B0005C29033022078000BA0B5F290800840AFA
:1002C00054292808A600A401A40A831603130112C6
:1002D0000000011683120313010826020319642982
:1002E000A409240AA70008000330BB0027308400BB
:1002F0000310800D840A800D840A800D840A800D0D
:10030000BB0B762908008316031332308500831255
:100310000313D9212B1185182B15831603133030A5
:100320008500831203132B1D9729E5200800DC208C
:1003300008001030BE0012309F00831603133130C6
:10034000850083120313E121BE03A0303E0783160C
:1003500003139F0083120313E1211F1BB229003CEA
:10036000031DA4298312031307309F008316031370
:1003700030308500831203133E08093C031CC62954
:100380002030132130303E07132108003130132173
:1003900026303E0713210800A201A20FD029080031
:1003A000A30FD029CD29F030A400CC21A40FD5294A
:1003B0000800A201A20FDA290800D921D921D921E8
:1003C0000800DD21DD21DD21DD21DD21DD21DD2133
:1003D00008005730C000FC214E30C000FC213230F4
:1003E000C000FC214130C000FC210A30C000FC21CB
:1003F0000D30C000FC21080083160313483086002E
:1004000083120313861316220830A100C00C861332
:10041000031886171622A10B062A8617D9218316E0
:100420000313C83086008312031308006830A2004B
:08043000A20B182A08000800C5
:02400E00623F0F
:00000001FF
